:1000000012C02DC02BC02AC029C028C027C026C0BE
:1000100025C024C023C022C021C020C01FC01EC0D4
:100020001DC01CC01BC011241FBECFE5D4E0DEBF25
:10003000CDBF10E0A0E6B0E0EEEDF9E102C0059022
:100040000D92A837B107D9F710E0A8E7B0E001C0DA
:100050001D92AC39B107E1F7CED8BFCCD1CF1F92FA
:100060000F920FB60F9211242F933F934F938F93BC
:100070009F93C59A80917B00882329F080917C0012
:100080008F5F80937C0080917D008F5F80937D00E7
:1000900080917D008F3F29F48BB78F7B8BBFA89A0F
:1000A000E1C68AB780648ABF9091600080917B002E
:1000B000882321F080917C0082FD906C97FF02C024
:1000C000A89A01C0A898492F440F90E820E030E09A
:1000D000999BB7C60AB606FCE4CF999BB2C60AB68E
:1000E00006FCDFCF999BADC60AB606FCDACF999B1A
:1000F000A8C60AB606FCD5CF999BA3C60AB606FCCD
:10010000D0CF999B9EC60AB606FCCBCF999B99C6C9
:100110000AB606FCC6CF999B94C60AB606FCC1CFA8
:10012000999B8FC60AB606FCBCCF999B8AC60AB6B5
:1001300006FCB7CF999B85C60AB606FCB2CF999B41
:1001400080C60AB606FCADCF999B7BC60AB606FCF4
:10015000A8CF999B76C60AB606FCA3CF999B71C619
:100160000AB606FC9ECF999B6CC60AB606FC99CFD0
:10017000999B67C60AB606FC94CF999B62C60AB6DD
:1001800006FC8FCF999B5DC60AB606FC8ACF999B69
:1001900058C60AB606FC85CF999B53C60AB606FC1C
:1001A00080CF999B4EC60AB606FC7BCF999B49C669
:1001B0000AB606FC76CF999B44C60AB606FC71CFF8
:1001C000999B3FC60AB606FC6CCF999B3AC60AB605
:1001D00006FC67CF999B35C60AB606FC62CF999B91
:1001E00030C60AB606FC5DCF999B2BC60AB606FC44
:1001F00058CF999B26C60AB606FC53CF999B21C6B9
:100200000AB606FC4ECF999B1CC60AB606FC49CF1F
:10021000999B17C60AB606FC44CF999B12C60AB62C
:1002200006FC3FCF999B0DC60AB606FC3ACF999BB8
:1002300008C60AB606FC35CF999B03C60AB606FC6B
:1002400030CF999BFEC50AB606FC2BCF999BF9C50A
:100250000AB606FC26CF999BF4C50AB606FC21CF48
:10026000999BEFC50AB606FC1CCF999BEAC50AB656
:1002700006FC17CF999BE5C50AB606FC12CF999BE1
:10028000E0C50AB606FC0DCF999BDBC50AB606FC95
:1002900008CF999BD6C50AB606FC03CF999BD1C55A
:1002A0000AB606FCFECE999BCCC50AB606FCF9CE72
:1002B000999BC7C50AB606FCF4CE999BC2C50AB67F
:1002C00006FCEFCE999BBDC50AB606FCEACE999B0B
:1002D000B8C50AB606FCE5CE999BB3C50AB606FCBE
:1002E000E0CE999BAEC50AB606FCDBCE999BA9C5AC
:1002F0000AB606FCD6CE999BA4C50AB606FCD1CE9A
:10030000999B9FC50AB606FCCCCE999B9AC50AB6A6
:1003100006FCC7CE999B95C50AB606FCC2CE999B32
:1003200090C50AB606FCBDCE999B8BC50AB606FCE5
:10033000B8CE999B86C50AB606FCB3CE999B81C5FB
:100340000AB606FCAECE999B7CC50AB606FCA9CEC1
:10035000999B77C50AB606FCA4CE999B72C50AB6CE
:1003600006FC9FCE999B6DC50AB606FC9ACE999B5A
:1003700068C50AB606FC95CE999B63C50AB606FC0D
:1003800090CE999B5EC50AB606FC8BCE999B59C54B
:100390000AB606FC86CE999B54C50AB606FC81CEE9
:1003A000999B4FC50AB606FC7CCE999B4AC50AB6F6
:1003B00006FC77CE999B45C50AB606FC72CE999B82
:1003C00040C50AB606FC6DCE999B3BC50AB606FC35
:1003D00068CE999B36C50AB606FC63CE999B31C59B
:1003E0000AB606FC5ECE999B2CC50AB606FC59CE11
:1003F000999B27C50AB606FC54CE999B22C50AB61E
:1004000006FC4FCE999B1DC50AB606FC4ACE999BA9
:1004100018C50AB606FC45CE999B13C50AB606FC5C
:1004200040CE999B0EC50AB606FC3BCE999B09C5EA
:100430000AB606FC36CE999B04C50AB606FC31CE38
:10044000999BFFC40AB606FC2CCE999BFAC40AB647
:1004500006FC27CE999BF5C40AB606FC22CE999BD2
:10046000F0C40AB606FC1DCE999BEBC40AB606FC86
:1004700018CE999BE6C40AB606FC13CE999BE1C43C
:100480000AB606FC0ECE999BDCC40AB606FC09CE61
:10049000999BD7C40AB606FC04CE999BD2C40AB66F
:1004A00006FCFFCD999BCDC40AB606FCFACD999BFC
:1004B000C8C40AB606FCF5CD999BC3C40AB606FCAF
:1004C000F0CD999BBEC40AB606FCEBCD999BB9C48E
:1004D0000AB606FCE6CD999BB4C40AB606FCE1CD8B
:1004E000999BAFC40AB606FCDCCD999BAAC40AB698
:1004F00006FCD7CD999BA5C40AB606FCD2CD999B24
:10050000A0C40AB606FCCDCD999B9BC40AB606FCD6
:10051000C8CD999B96C40AB606FCC3CD999B91C4DD
:100520000AB606FCBECD999B8CC40AB606FCB9CDB2
:10053000999B87C40AB606FCB4CD999B82C40AB6BF
:1005400006FCAFCD999B7DC40AB606FCAACD999B4B
:1005500078C40AB606FCA5CD999B73C40AB606FCFE
:10056000A0CD999B6EC40AB606FC9BCD999B69C42D
:100570000AB606FC96CD999B64C40AB606FC91CDDA
:10058000999B5FC40AB606FC8CCD999B5AC40AB6E7
:1005900006FC87CD999B55C40AB606FC82CD999B73
:1005A00050C40AB606FC7DCD999B4BC40AB606FC26
:1005B00078CD999B46C40AB606FC73CD999B41C47D
:1005C0000AB606FC6ECD999B3CC40AB606FC69CD02
:1005D000999B37C40AB606FC64CD999B32C40AB60F
:1005E00006FC5FCD999B2DC40AB606FC5ACD999B9B
:1005F00028C40AB606FC55CD999B23C40AB606FC4E
:1006000050CD999B1EC40AB606FC4BCD999B19C4CC
:100610000AB606FC46CD999B14C40AB606FC41CD29
:10062000999B0FC40AB606FC3CCD999B0AC40AB636
:1006300006FC37CD999B05C40AB606FC32CD999BC2
:1006400000C40AB606FC2DCD999BFBC30AB606FC76
:1006500028CD999BF6C30AB606FC23CD999BF1C31E
:100660000AB606FC1ECD999BECC30AB606FC19CD52
:10067000999BE7C30AB606FC14CD999BE2C30AB660
:1006800006FC0FCD999BDDC30AB606FC0ACD999BEB
:10069000D8C30AB606FC05CD999BD3C30AB606FC9F
:1006A00000CD999BCEC30AB606FCFBCC999BC9C36F
:1006B0000AB606FCF6CC999BC4C30AB606FCF1CC7C
:1006C000999BBFC30AB606FCECCC999BBAC30AB689
:1006D00006FCE7CC999BB5C30AB606FCE2CC999B15
:1006E000B0C30AB606FCDDCC999BABC30AB606FCC8
:1006F000D8CC999BA6C30AB606FCD3CC999BA1C3C0
:100700000AB606FCCECC999B9CC30AB606FCC9CCA3
:10071000999B97C30AB606FCC4CC999B92C30AB6B0
:1007200006FCBFCC999B8DC30AB606FCBACC999B3C
:1007300088C30AB606FCB5CC999B83C30AB606FCEF
:10074000B0CC999B7EC30AB606FCABCC999B79C30F
:100750000AB606FCA6CC999B74C30AB606FCA1CCCB
:10076000999B6FC30AB606FC9CCC999B6AC30AB6D8
:1007700006FC97CC999B65C30AB606FC92CC999B64
:1007800060C30AB606FC8DCC999B5BC30AB606FC17
:1007900088CC999B56C30AB606FC83CC999B51C35F
:1007A0000AB606FC7ECC999B4CC30AB606FC79CCF3
:1007B000999B47C30AB606FC74CC999B42C30AB600
:1007C00006FC6FCC999B3DC30AB606FC6ACC999B8C
:1007D00038C30AB606FC65CC999B33C30AB606FC3F
:1007E00060CC999B2EC30AB606FC5BCC999B29C3AF
:1007F0000AB606FC56CC999B24C30AB606FC51CC1B
:10080000999B1FC30AB606FC4CCC999B1AC30AB627
:1008100006FC47CC999B15C30AB606FC42CC999BB3
:1008200010C30AB606FC3DCC999B0BC30AB606FC66
:1008300038CC999B06C30AB606FC33CC999B01C3FE
:100840000AB606FC2ECC999BFCC20AB606FC29CC43
:10085000999BF7C20AB606FC24CC999BF2C20AB651
:1008600006FC1FCC999BEDC20AB606FC1ACC999BDC
:10087000E8C20AB606FC15CC999BE3C20AB606FC90
:1008800010CC999BDEC20AB606FC0BCC999BD9C250
:100890000AB606FC06CC999BD4C20AB606FC01CC6B
:1008A000999BCFC20AB606FCFCCB999BCAC20AB67A
:1008B00006FCF7CB999BC5C20AB606FCF2CB999B06
:1008C000C0C20AB606FCEDCB999BBBC20AB606FCB9
:1008D000E8CB999BB6C20AB606FCE3CB999BB1C2A2
:1008E0000AB606FCDECB999BACC20AB606FCD9CB95
:1008F000999BA7C20AB606FCD4CB999BA2C20AB6A2
:1009000006FCCFCB999B9DC20AB606FCCACB999B2D
:1009100098C20AB606FCC5CB999B93C20AB606FCE0
:10092000C0CB999B8EC20AB606FCBBCB999B89C2F1
:100930000AB606FCB6CB999B84C20AB606FCB1CBBC
:10094000999B7FC20AB606FCACCB999B7AC20AB6C9
:1009500006FCA7CB999B75C20AB606FCA2CB999B55
:1009600070C20AB606FC9DCB999B6BC20AB606FC08
:1009700098CB999B66C20AB606FC93CB999B61C241
:100980000AB606FC8ECB999B5CC20AB606FC89CBE4
:10099000999B57C20AB606FC84CB999B52C20AB6F1
:1009A00006FC7FCB999B4DC20AB606FC7ACB999B7D
:1009B00048C20AB606FC75CB999B43C20AB606FC30
:1009C00070CB999B3EC20AB606FC6BCB999B39C291
:1009D0000AB606FC66CB999B34C20AB606FC61CB0C
:1009E000999B2FC20AB606FC5CCB999B2AC20AB619
:1009F00006FC57CB999B25C20AB606FC52CB999BA5
:100A000020C20AB606FC4DCB999B1BC20AB606FC57
:100A100048CB999B16C20AB606FC43CB999B11C2E0
:100A20000AB606FC3ECB999B0CC20AB606FC39CB33
:100A3000999B07C20AB606FC34CB999B02C20AB640
:100A400006FC2FCB999BFDC10AB606FC2ACB999BCD
:100A5000F8C10AB606FC25CB999BF3C10AB606FC81
:100A600020CB999BEEC10AB606FC1BCB999BE9C132
:100A70000AB606FC16CB999BE4C10AB606FC11CB5C
:100A8000999BDFC10AB606FC0CCB999BDAC10AB66A
:100A900006FC07CB999BD5C10AB606FC02CB999BF5
:100AA000D0C10AB606FCFDCA999BCBC10AB606FCAA
:100AB000F8CA999BC6C10AB606FCF3CA999BC1C184
:100AC0000AB606FCEECA999BBCC10AB606FCE9CA86
:100AD000999BB7C10AB606FCE4CA999BB2C10AB693
:100AE00006FCDFCA999BADC10AB606FCDACA999B1F
:100AF000A8C10AB606FCD5CA999BA3C10AB606FCD2
:100B0000D0CA999B9EC10AB606FCCBCA999B99C1D3
:100B10000AB606FCC6CA999B94C10AB606FCC1CAAD
:100B2000999B8FC10AB606FCBCCA999B8AC10AB6BA
:100B300006FCB7CA999B85C10AB606FCB2CA999B46
:100B400080C10AB606FCADCA999B7BC10AB606FCF9
:100B5000A8CA999B76C10AB606FCA3CA999B71C123
:100B60000AB606FC9ECA999B6CC10AB606FC99CAD5
:100B7000999B67C10AB606FC94CA999B62C10AB6E2
:100B800006FC8FCA999B5DC10AB606FC8ACA999B6E
:100B900058C10AB606FC85CA999B53C10AB606FC21
:100BA00080CA999B4EC10AB606FC7BCA999B49C173
:100BB0000AB606FC76CA999B44C10AB606FC71CAFD
:100BC000999B3FC10AB606FC6CCA999B3AC10AB60A
:100BD00006FC67CA999B35C10AB606FC62CA999B96
:100BE00030C10AB606FC5DCA999B2BC10AB606FC49
:100BF00058CA999B26C10AB606FC53CA999B21C1C3
:100C00000AB606FC4ECA999B1CC10AB606FC49CA24
:100C1000999B17C10AB606FC44CA999B12C10AB631
:100C200006FC3FCA999B0DC10AB606FC3ACA999BBD
:100C300008C10AB606FC35CA999B03C10AB606FC70
:100C400030CA999BFEC00AB606FC2BCA999BF9C014
:100C50000AB606FC26CA999BF4C00AB606FC21CA4D
:100C6000999BEFC00AB606FC1CCA999BEAC00AB65B
:100C700006FC17CA999BE5C00AB606FC12CA999BE6
:100C8000E0C00AB606FC0DCA999BDBC00AB606FC9A
:100C900008CA999BD6C00AB606FC03CA999BD1C064
:100CA0000AB606FCFEC9999BCCC00AB606FCF9C977
:100CB000999BC7C00AB606FCF4C9999BC2C00AB684
:100CC00006FCEFC9999BBDC00AB606FCEAC9999B10
:100CD000B8C00AB606FCE5C9999BB3C00AB606FCC3
:100CE000E0C9999BAEC00AB606FCDBC9999BA9C0B6
:100CF0000AB606FCD6C9999BA4C00AB606FCD1C99F
:100D0000999B9FC00AB606FCCCC9999B9AC00AB6AB
:100D100006FCC7C9999B95C00AB606FCC2C9999B37
:100D200090C00AB606FCBDC9999B8BC00AB606FCEA
:100D3000B8C9999B86C00AB606FCB3C9999B81C005
:100D40000AB606FCAEC9999B7CC00AB606FCA9C9C6
:100D5000999B77C00AB606FCA4C9999B72C00AB6D3
:100D600006FC9FC9999B6DC00AB606FC9AC9999B5F
:100D700068C00AB606FC95C9999B63C00AB606FC12
:100D800090C9999B5EC00AB606FC8BC9999B59C055
:100D90000AB606FC86C9999B54C00AB606FC81C9EE
:100DA000999B4FC00AB606FC7CC9999B4AC00AB6FB
:100DB00006FC77C9999B45C00AB606FC72C9999B87
:100DC00040C00AB606FC6DC9999B3BC00AB606FC3A
:100DD00068C9999B36C00AB606FC63C9999B31C0A5
:100DE0000AB606FC5EC9999B2CC00AB606FC59C916
:100DF000999B27C00AB606FC54C9999B22C00AB623
:100E000006FC4FC9999B1DC00AB606FC4AC9999BAE
:100E100018C00AB606FC45C9999B13C00AB606FC61
:100E200040C9999B0EC00AB606FC3BC9999B09C0F4
:100E30000AB606FC36C9999B04C00AB606FC31C93D
:100E40000DC0892F842311F0A89A01C0A898969507
:100E50002F5F3F4F2830310509F03AC981E0809378
:100E60007A00C5989F918F914F913F912F910F904C
:100E70000FBE0F901F901895482F90E820E030E0AB
:100E8000FB01E20FF31F892F8423808396952F5F48
:100E90003F4F28303105A1F70895992787FD909598
:100EA000A92FB92FBC01CD0120EC3DE540E050E079
:100EB0002BD52FEF3FE740E050E045D5822F089536
:100EC000892B71F02091600080E890E002C0959538
:100ED00087956A95E2F78095822380936000089554
:100EE0002091600080E890E002C0959587956A9512
:100EF000E2F7282B209360000895EF92FF920F9362
:100F00001F93CF93DF937A01082F10E0C22FD0E018
:100F100080E890E08C1B9D0B081719071CF481E0FA
:100F200090E0CEDFC058DF4FC017D10724F481E036
:100F300090E0B701C5DFDF91CF911F910F91FF9036
:100F4000EF9008959F92AF92BF92CF92DF92EF926F
:100F5000FF920F931F93CF93DF935A0169019E2C49
:100F6000E82EFF2410E0C0E8D0E0CE01801B910BFA
:100F7000E816F90664F481E090E0A2DFC919D1090E
:100F8000EC16FD0624F481E090E0B60199DF0058EC
:100F90001F4F0E151F057CF481E090E0B50190DF36
:100FA000892D90E080589F4F8E159F0524F481E095
:100FB00090E0B60185DFDF91CF911F910F91FF90F7
:100FC000EF90DF90CF90BF90AF909F900895EF92F9
:100FD0000F9380917800909179008130910509F408
:100FE00057C08230910509F4A4C0892B09F0F6C0DE
:100FF00080919A0090E08071907060E070E060DF16
:1010000080919A0090E08870907061E070E058DF05
:1010100080919A0090E08078907062E070E050DFFC
:1010200080919A0090E08170907063E070E048DFFA
:1010300080919B0090E08170907064E070E040DFF0
:1010400080919B0090E08270907065E070E038DFE6
:1010500080919B0090E08870907066E070E030DFD7
:1010600080919B0090E08470907067E070E028DFD2
:101070008091940066E070E047E050E028E33DDFB7
:101080008091950064E070E045E050E028E34FC0B7
:1010900080919A0090E08071907060E070E010DFC5
:1010A00080919A0090E08870907061E070E008DFB5
:1010B00080919A0090E08078907062E070E000DFAC
:1010C00080919A0090E08170907063E070E0F8DEAB
:1010D00080919B0090E08170907064E070E0F0DEA1
:1010E00080919B0090E08270907065E070E0E8DE97
:1010F00080919B0090E08870907066E070E0E0DE88
:1011000080919B0090E08470907067E070E0D8DE82
:101110008091940066E070E047E050E020E2EDDE70
:101120008091950064E070E045E050E020E2E5DE6B
:1011300055C080919A0090E08071907060E070E0FE
:10114000BFDE80919A0090E08870907061E070E05E
:10115000B7DE80919A0090E08078907062E070E055
:10116000AFDE80919A0090E08170907063E070E053
:10117000A7DE80919B0090E08170907064E070E049
:101180009FDE80919B0090E08270907065E070E03F
:1011900097DE80919B0090E08870907066E070E030
:1011A0008FDE80919B0090E08470907067E070E02B
:1011B00087DE8091940066E070E047E050E021E037
:1011C00030E000E290E4E92EBDDE8091950064E01D
:1011D00070E045E050E021E030E0B4DE80919A001C
:1011E00085FF04C081E080937B0002C010927B00E9
:1011F0000F91EF90089583D0FC019093930080931A
:10120000920011BA9FEF92BB17BA98BB80E287BBDE
:10121000C59881E084BB95BB85B7836085BF8BB7DC
:1012200080648BBF8BB78F778BBF0284F385E02DF3
:10123000099588E893E120E931E0F9013197F1F768
:101240000197D9F7E0919200F09193000484F5851D
:10125000E02D0995E0919200F09193000088F189CA
:10126000E02D84E990E0099580919A00282F84FF71
:1012700006C082E090E0909379008093780023FF8D
:1012800006C081E090E09093790080937800ECD2E2
:10129000789480917A00882321F010927A00F2D21B
:1012A000C5981FD3882321F480917D008F3F89F753
:1012B000E0919200F09193000484F585E02D09956A
:1012C000E0919200F09193000684F785E02D099556
:1012D000882359F0E0919200F09193000088F18901
:1012E000E02D84E990E0099572DE80917D008F3FCA
:1012F00019F48BB780648BBF10927D00CACF81E652
:1013000090E00895009741F0DC01EEE7F0E088E01E
:1013100001900D928150E1F7A6E8B0E0EEE7F0E031
:1013200088E001900D928150E1F708958091750059
:1013300090917600892B31F0109276001092750012
:1013400081E008958EE790E066E870E048E050E0C4
:1013500037D308950F931F93DF93CF93CDB7DEB7A5
:10136000C850D1400FB6F894DEBF0FBECDBF80E0AD
:10137000E3D1FE01399680E0EF93FF9300E810E49B
:101380001023A9F00000A59A000000000000000052
:10139000000000000000000000000000A59838E0F8
:1013A0003A95F1F700000000069561F0E8CFA59AA4
:1013B0003BE03A95F1F70000A59800000000069583
:1013C00009F0DDCFA59800E813E01023A9F0000094
:1013D000A59A0000000000000000000000000000CE
:1013E000000000000000A59838E03A95F1F70000F1
:1013F0000000069561F0E8CFA59A3BE03A95F1F739
:101400000000A59800000000069509F0DDCFA59822
:1014100000E8182F1023A9F00000A59A0000000092
:1014200000000000000000000000000000000000BC
:10143000A59838E03A95F1F700000000069561F0B4
:10144000E8CFA59A3BE03A95F1F70000A598000097
:101450000000069509F0DDCFA5980000000000000F
:101460000000A59A0000000000000000A59813B33A
:101470001072E9F330E40FE30A9519F013B3107218
:10148000D9F788278095FF91EF91C198EF93FF934B
:10149000882700270395B1F09D99FCCFC19808C01B
:1014A0000027039579F09D99FCCF839551F0019326
:1014B0000027039539F09D9BFCCF839511F0019394
:1014C000EFCFC19AFF91EF91813821F081E08093B5
:1014D0008E0012C1DF01AE0147575F4F20E09081BF
:1014E0008181981708F421E02D933296E417F507CF
:1014F000A9F7FE01319688E0DF011D928A95E9F790
:101500004981FE01799620E030E060E870E080815A
:10151000882339F0CB01022E02C0959587950A9455
:10152000E2F7482B2F5F3F4F31962830310579F78E
:1015300049834A81FE01B19620E030E060E870E026
:101540008081882339F0CB01022E02C095958795C2
:101550000A94E2F7482B2F5F3F4F31962830310530
:1015600079F740954A834B81FE01B99620E030E03F
:1015700060E870E08081882339F0CB01022E02C040
:10158000959587950A94E2F7482B2F5F3F4F319648
:101590002830310579F74B834C81FE01F19620E02C
:1015A00030E060E870E08081882311F080E007C0BF
:1015B000CB01022E02C0959587950A94E2F7482B3D
:1015C0002F5F3F4F31962830310569F74C834D81AD
:1015D000FE01F99620E030E060E870E08081882329
:1015E00039F0CB01022E02C0959587950A94E2F757
:1015F000482B2F5F3F4F31962830310579F74095C2
:101600004D834E81FE01EF5BFF4F20E030E060E84C
:1016100070E08081882339F0CB01022E02C09595BD
:1016200087950A94E2F7482B2F5F3F4F3196283079
:10163000310579F740954E834F81FE013C9620E0BD
:1016400030E061E070E08081882339F0CB01022E28
:1016500002C0880F991F0A94E2F7482B2F5F3F4F73
:1016600031962530310579F7FE01729620E030E0A1
:1016700060E270E08081882339F0CB01022E02C045
:10168000880F991F0A94E2F7482B2F5F3F4F31963E
:101690002330310579F74F834885FE01759620E0A8
:1016A00030E061E070E08081882339F0CB01022EC8
:1016B00002C0880F991F0A94E2F7482B2F5F3F4F13
:1016C00031962430310579F7898180937E008A81B3
:1016D00080937F008B81809380008C818093810038
:1016E0008D81809382008E81809383008F8180938F
:1016F00084004093850080E0C85FDE4F0FB6F89409
:10170000DEBF0FBECDBFCF91DF911F910F91089526
:1017100010928E001FDE90E080918E00882309F4E5
:1017200091E0892F08958FB7F894B99AC198A59838
:10173000AD988FBF0FDE08950F931F93DF93CF9364
:10174000CDB7DEB7C254D0400FB6F894DEBF0FBE9F
:10175000CDBFFE013296982FEF93FF9300E8192F2B
:101760001023D1F0000068C0A59A0000000000001E
:101770000000000000000000000000000000000069
:10178000000000000000A5983CE03A95F1F7000049
:101790000000069581F0E3CFA59A3FE03A95F1F776
:1017A0000000A598000000000000000000000000FC
:1017B000069509F0D4CFA5980000000000000000B5
:1017C0000000000000000000A59A000000000000DA
:1017D0000000000000000000000000000000000009
:1017E000000000000000A59830E20FEF0A9511F10B
:1017F00013B31072D9F700000000000000000000D1
:1018000000000000000000000000000000000000D8
:101810000000000023B3207221933A9539F00FEFB6
:101820000A9541F023B3207201F7FACF882704C04C
:10183000832F02C088278095FF91EF91898389814A
:101840008F3F19F020E030E002C02FEF3FEFC901D9
:10185000CE5BDF4F0FB6F894DEBF0FBECDBFCF918A
:10186000DF911F910F9108951FBC83E08EBD1DBCB9
:101870001CBC109291008DE199E0909390008093B0
:101880008F00089508B602FE04C088B7846088BF40
:101890001AC08CB59DB526E0853A9207D0F02AE0B3
:1018A0008C38920718F0875E934002C08DE199E072
:1018B0009093900080938F0080918F009091900082
:1018C000845A964030F48DE199E090939000809393
:1018D0008F001DBC1CBC88B7846088BF109291002B
:1018E000089580919100882369F42CB53DB58091CD
:1018F0008F00909190002817390720F081E08093A5
:101900009100089580E00895629FD001739FF001D7
:10191000829FE00DF11D649FE00DF11D929FF00D7F
:10192000839FF00D749FF00D659FF00D9927729FB6
:10193000B00DE11DF91F639FB00DE11DF91FBD0141
:10194000CF011124089597FB092E05260ED057FDCF
:1019500004D014D00AD0001C38F45095409530952E
:1019600021953F4F4F4F5F4F0895F6F79095809523
:10197000709561957F4F8F4F9F4F0895A1E21A2E6A
:10198000AA1BBB1BFD010DC0AA1FBB1FEE1FFF1F23
:10199000A217B307E407F50720F0A21BB30BE40B73
:1019A000F50B661F771F881F991F1A9469F76095BA
:1019B0007095809590959B01AC01BD01CF01089574
:1019C000FB01DC0104C08D910190801921F441508C
:0E19D0005040C8F7881B990B0895F894FFCF7C
:1019DE00FF08000000000000000000930BAA09960B
:0819EE00098209880B010000C9
:00000001FF
